 getfldecl004

 Timestamp is 71680712 (reproducible build file hash)

 Preferred load address is 0000000180000000

 Start         Length     Name                   Class
 0001:00000000 00002b40H .text$mn                CODE
 0001:00002b40 00000036H .text$mn$00             CODE
 0001:00002b76 00000092H .text$x                 CODE
 0002:00000000 00000198H .idata$5                DATA
 0002:00000198 00000038H .00cfg                  DATA
 0002:000001d0 00000008H .CRT$XCA                DATA
 0002:000001d8 00000008H .CRT$XCZ                DATA
 0002:000001e0 00000008H .CRT$XIA                DATA
 0002:000001e8 00000008H .CRT$XIC                DATA
 0002:000001f0 00000008H .CRT$XIZ                DATA
 0002:000001f8 00000008H .CRT$XLA                DATA
 0002:00000200 00000008H .CRT$XLZ                DATA
 0002:00000208 00000008H .CRT$XPA                DATA
 0002:00000210 00000008H .CRT$XPZ                DATA
 0002:00000218 00000008H .CRT$XTA                DATA
 0002:00000220 00000010H .CRT$XTZ                DATA
 0002:00000228 00000000H .gehcont$y              DATA
 0002:00000228 00000000H .gfids$y                DATA
 0002:00000230 00001bd0H .rdata                  DATA
 0002:00001e00 00000000H .rdata$CastGuardVftablesA DATA
 0002:00001e00 00000000H .rdata$CastGuardVftablesC DATA
 0002:00001e00 00000028H .rdata$T                DATA
 0002:00001e28 000000a4H .rdata$voltmd           DATA
 0002:00001ecc 0000031cH .rdata$zzzdbg           DATA
 0002:000021e8 00000008H .rtc$IAA                DATA
 0002:000021f0 00000008H .rtc$IZZ                DATA
 0002:000021f8 00000008H .rtc$TAA                DATA
 0002:00002200 00000008H .rtc$TZZ                DATA
 0002:00002208 00000004H .tls                    DATA
 0002:0000220c 00000004H .tls$                   DATA
 0002:00002210 00000008H .tls$ZZZ                DATA
 0002:00002218 000002e8H .xdata                  DATA
 0002:00002500 000003ecH .edata                  DATA
 0002:000028ec 00000064H .idata$2                DATA
 0002:00002950 00000018H .idata$3                DATA
 0002:00002968 00000198H .idata$4                DATA
 0002:00002b00 0000041eH .idata$6                DATA
 0003:00000000 000001a0H .data                   DATA
 0003:000001a0 0001b238H .bss                    DATA
 0004:00000000 00000378H .pdata                  DATA

  Address         Publics by Value              Rva+Base               Lib:Object

 0000:00000000       __AbsoluteZero             0000000000000000     <absolute>
 0000:00000000       ___safe_se_handler_count   0000000000000000     <absolute>
 0000:00000000       ___safe_se_handler_table   0000000000000000     <absolute>
 0000:00000000       __arm64x_extra_rfe_table   0000000000000000     <absolute>
 0000:00000000       __arm64x_extra_rfe_table_size 0000000000000000     <absolute>
 0000:00000000       __arm64x_native_entrypoint 0000000000000000     <absolute>
 0000:00000000       __arm64x_redirection_metadata 0000000000000000     <absolute>
 0000:00000000       __arm64x_redirection_metadata_count 0000000000000000     <absolute>
 0000:00000000       __dynamic_value_reloc_table 0000000000000000     <absolute>
 0000:00000000       __enclave_config           0000000000000000     <absolute>
 0000:00000000       __guard_check_icall_a64n_fptr 0000000000000000     <absolute>
 0000:00000000       __guard_eh_cont_count      0000000000000000     <absolute>
 0000:00000000       __guard_eh_cont_table      0000000000000000     <absolute>
 0000:00000000       __guard_fids_count         0000000000000000     <absolute>
 0000:00000000       __guard_fids_table         0000000000000000     <absolute>
 0000:00000000       __guard_iat_count          0000000000000000     <absolute>
 0000:00000000       __guard_iat_table          0000000000000000     <absolute>
 0000:00000000       __guard_longjmp_count      0000000000000000     <absolute>
 0000:00000000       __guard_longjmp_table      0000000000000000     <absolute>
 0000:00000000       __hybrid_auxiliary_iat     0000000000000000     <absolute>
 0000:00000000       __hybrid_auxiliary_iat_copy 0000000000000000     <absolute>
 0000:00000000       __hybrid_code_map          0000000000000000     <absolute>
 0000:00000000       __hybrid_code_map_count    0000000000000000     <absolute>
 0000:00000000       __x64_code_ranges_to_entry_points 0000000000000000     <absolute>
 0000:00000000       __x64_code_ranges_to_entry_points_count 0000000000000000     <absolute>
 0000:00000100       __guard_flags              0000000000000100     <absolute>
 0000:00000000       __ImageBase                0000000180000000     <linker-defined>
 0001:00000000       ?NewObject@JNIEnv_@@QEAAPEAV_jobject@@PEAV_jclass@@PEAU_jmethodID@@ZZ 0000000180001000 f i libgetfldecl004.obj
 0001:00000028       ?TranslateError@@YAPEBDW4jvmtiError@@@Z 0000000180001028 f   libgetfldecl004.obj
 0001:000002e0       ?nsk_jni_check_exception@@YAHPEAUJNIEnv_@@QEBDH@Z 00000001800012e0 f   libgetfldecl004.obj
 0001:00000424       ?nsk_jni_lverify@@YAHHPEAUJNIEnv_@@HQEBDH1ZZ 0000000180001424 f   libgetfldecl004.obj
 0001:000004c4       Agent_Initialize           00000001800014c4 f   libgetfldecl004.obj
 0001:00000538       Agent_OnAttach             0000000180001538 f   libgetfldecl004.obj
 0001:00000538       Agent_OnLoad               0000000180001538 f   libgetfldecl004.obj
 0001:00000540       Java_nsk_jvmti_GetFieldDeclaringClass_getfldecl004_check 0000000180001540 f   libgetfldecl004.obj
 0001:000006c8       Java_nsk_jvmti_GetFieldDeclaringClass_getfldecl004_getRes 00000001800016c8 f   libgetfldecl004.obj
 0001:000006d0       Java_nsk_jvmti_unit_FollowReferences_FollowRefObjects_addRefToVerify 00000001800016d0 f   libgetfldecl004.obj
 0001:000008a8       Java_nsk_jvmti_unit_FollowReferences_FollowRefObjects_getTag 00000001800018a8 f   libgetfldecl004.obj
 0001:00000968       Java_nsk_jvmti_unit_FollowReferences_FollowRefObjects_resetRefsToVerify 0000000180001968 f   libgetfldecl004.obj
 0001:00000970       Java_nsk_jvmti_unit_FollowReferences_FollowRefObjects_resetTags 0000000180001970 f   libgetfldecl004.obj
 0001:000009b4       Java_nsk_jvmti_unit_FollowReferences_FollowRefObjects_setTag 00000001800019b4 f   libgetfldecl004.obj
 0001:00000c0c       Java_nsk_share_jvmti_ArgumentHandler_getAgentOptionsString 0000000180001c0c f   libgetfldecl004.obj
 0001:00000cbc       Java_nsk_share_jvmti_DebugeeClass_checkStatus 0000000180001cbc f   libgetfldecl004.obj
 0001:00000d44       Java_nsk_share_jvmti_DebugeeClass_resetAgentData 0000000180001d44 f   libgetfldecl004.obj
 0001:00000da4       Java_nsk_share_jvmti_RedefineAgent_agentStatus 0000000180001da4 f   libgetfldecl004.obj
 0001:00000db0       Java_nsk_share_jvmti_RedefineAgent_isRedefined 0000000180001db0 f   libgetfldecl004.obj
 0001:00000dbc       Java_nsk_share_jvmti_RedefineAgent_redefineAttempted 0000000180001dbc f   libgetfldecl004.obj
 0001:00000dc8       MA_checkStatus             0000000180001dc8 f   libgetfldecl004.obj
 0001:00000e6c       __local_stdio_printf_options 0000000180001e6c f i libgetfldecl004.obj
 0001:0000104c       exitOnError                000000018000204c f   libgetfldecl004.obj
 0001:00001100       fprintf                    0000000180002100 f i libgetfldecl004.obj
 0001:00001144       nsk_jvmti_lverify          0000000180002144 f   libgetfldecl004.obj
 0001:00001234       nsk_jvmti_resetAgentData   0000000180002234 f   libgetfldecl004.obj
 0001:000012b4       nsk_jvmti_setFailStatus    00000001800022b4 f   libgetfldecl004.obj
 0001:000012f0       nsk_lcomplain              00000001800022f0 f   libgetfldecl004.obj
 0001:00001310       nsk_ldisplay               0000000180002310 f   libgetfldecl004.obj
 0001:00001330       nsk_ltrace                 0000000180002330 f   libgetfldecl004.obj
 0001:00001350       nsk_lvcomplain             0000000180002350 f   libgetfldecl004.obj
 0001:00001508       nsk_lvdisplay              0000000180002508 f   libgetfldecl004.obj
 0001:00001554       nsk_lverify                0000000180002554 f   libgetfldecl004.obj
 0001:000015b0       nsk_lvtrace                00000001800025b0 f   libgetfldecl004.obj
 0001:00001610       nsk_printf                 0000000180002610 f   libgetfldecl004.obj
 0001:00001638       nsk_vprintf                0000000180002638 f   libgetfldecl004.obj
 0001:000016ec       printf                     00000001800026ec f i libgetfldecl004.obj
 0001:00001c14       __raise_securityfailure    0000000180002c14 f   MSVCRT:gs_report.obj
 0001:00001c48       __report_gsfailure         0000000180002c48 f   MSVCRT:gs_report.obj
 0001:00001e88       __GSHandlerCheck           0000000180002e88 f   MSVCRT:gshandler.obj
 0001:00001ea8       __GSHandlerCheckCommon     0000000180002ea8 f   MSVCRT:gshandler.obj
 0001:00001f20       __security_check_cookie    0000000180002f20 f   MSVCRT:amdsecgs.obj
 0001:00002260       _DllMainCRTStartup         0000000180003260 f   MSVCRT:dll_dllmain.obj
 0001:000022a0       __scrt_acquire_startup_lock 00000001800032a0 f   MSVCRT:utility.obj
 0001:000022dc       __scrt_dllmain_after_initialize_c 00000001800032dc f   MSVCRT:utility.obj
 0001:00002310       __scrt_dllmain_before_initialize_c 0000000180003310 f   MSVCRT:utility.obj
 0001:00002328       __scrt_dllmain_crt_thread_attach 0000000180003328 f   MSVCRT:utility.obj
 0001:00002350       __scrt_dllmain_crt_thread_detach 0000000180003350 f   MSVCRT:utility.obj
 0001:00002368       __scrt_dllmain_exception_filter 0000000180003368 f   MSVCRT:utility.obj
 0001:000023c8       __scrt_dllmain_uninitialize_c 00000001800033c8 f   MSVCRT:utility.obj
 0001:000023f8       __scrt_dllmain_uninitialize_critical 00000001800033f8 f   MSVCRT:utility.obj
 0001:0000240c       __scrt_initialize_crt      000000018000340c f   MSVCRT:utility.obj
 0001:00002458       __scrt_initialize_onexit_tables 0000000180003458 f   MSVCRT:utility.obj
 0001:000024e4       __scrt_is_nonwritable_in_current_image 00000001800034e4 f   MSVCRT:utility.obj
 0001:0000257c       __scrt_release_startup_lock 000000018000357c f   MSVCRT:utility.obj
 0001:000025a0       __scrt_uninitialize_crt    00000001800035a0 f   MSVCRT:utility.obj
 0001:000025cc       _onexit                    00000001800035cc f   MSVCRT:utility.obj
 0001:00002608       atexit                     0000000180003608 f   MSVCRT:utility.obj
 0001:00002620       __crt_debugger_hook        0000000180003620 f   MSVCRT:utility_desktop.obj
 0001:00002628       __scrt_fastfail            0000000180003628 f   MSVCRT:utility_desktop.obj
 0001:00002774       _guard_check_icall_nop     0000000180003774 f i MSVCRT:guard_support.obj
 0001:00002778       __security_init_cookie     0000000180003778 f   MSVCRT:gs_support.obj
 0001:00002824       DllMain                    0000000180003824 f   MSVCRT:dll_dllmain_stub.obj
 0001:00002848       ?__scrt_initialize_type_info@@YAXXZ 0000000180003848 f   MSVCRT:tncleanup.obj
 0001:00002858       ?__scrt_uninitialize_type_info@@YAXXZ 0000000180003858 f   MSVCRT:tncleanup.obj
 0001:00002864       __local_stdio_scanf_options 0000000180003864 f i MSVCRT:default_local_stdio_options.obj
 0001:0000286c       __scrt_initialize_default_local_stdio_options 000000018000386c f   MSVCRT:default_local_stdio_options.obj
 0001:00002888       __scrt_get_dyn_tls_init_callback 0000000180003888 f   MSVCRT:dyn_tls_init.obj
 0001:00002890       _RTC_Initialize            0000000180003890 f   MSVCRT:initsect.obj
 0001:000028cc       _RTC_Terminate             00000001800038cc f   MSVCRT:initsect.obj
 0001:00002908       __isa_available_init       0000000180003908 f   MSVCRT:cpu_disp.obj
 0001:00002ab4       _get_startup_argv_mode     0000000180003ab4 f   MSVCRT:argv_mode.obj
 0001:00002abc       __scrt_is_ucrt_dll_in_use  0000000180003abc f   MSVCRT:ucrt_detection.obj
 0001:00002ad0       memcpy                     0000000180003ad0 f   vcruntime:VCRUNTIME140.dll
 0001:00002ad6       memset                     0000000180003ad6 f   vcruntime:VCRUNTIME140.dll
 0001:00002adc       strchr                     0000000180003adc f   vcruntime:VCRUNTIME140.dll
 0001:00002ae2       __C_specific_handler       0000000180003ae2 f   vcruntime:VCRUNTIME140.dll
 0001:00002ae8       __std_type_info_destroy_list 0000000180003ae8 f   vcruntime:VCRUNTIME140.dll
 0001:00002aee       strcmp                     0000000180003aee f   ucrt:api-ms-win-crt-string-l1-1-0.dll
 0001:00002af4       strlen                     0000000180003af4 f   ucrt:api-ms-win-crt-string-l1-1-0.dll
 0001:00002afa       _initterm                  0000000180003afa f   ucrt:api-ms-win-crt-runtime-l1-1-0.dll
 0001:00002b00       _initterm_e                0000000180003b00 f   ucrt:api-ms-win-crt-runtime-l1-1-0.dll
 0001:00002b06       _seh_filter_dll            0000000180003b06 f   ucrt:api-ms-win-crt-runtime-l1-1-0.dll
 0001:00002b0c       _configure_narrow_argv     0000000180003b0c f   ucrt:api-ms-win-crt-runtime-l1-1-0.dll
 0001:00002b12       _initialize_narrow_environment 0000000180003b12 f   ucrt:api-ms-win-crt-runtime-l1-1-0.dll
 0001:00002b18       _initialize_onexit_table   0000000180003b18 f   ucrt:api-ms-win-crt-runtime-l1-1-0.dll
 0001:00002b1e       _register_onexit_function  0000000180003b1e f   ucrt:api-ms-win-crt-runtime-l1-1-0.dll
 0001:00002b24       _execute_onexit_table      0000000180003b24 f   ucrt:api-ms-win-crt-runtime-l1-1-0.dll
 0001:00002b2a       _crt_atexit                0000000180003b2a f   ucrt:api-ms-win-crt-runtime-l1-1-0.dll
 0001:00002b30       _cexit                     0000000180003b30 f   ucrt:api-ms-win-crt-runtime-l1-1-0.dll
 0001:00002b38       __acrt_initialize          0000000180003b38 f   MSVCRT:ucrt_stubs.obj
 0001:00002b38       __acrt_thread_attach       0000000180003b38 f   MSVCRT:ucrt_stubs.obj
 0001:00002b38       __acrt_thread_detach       0000000180003b38 f   MSVCRT:ucrt_stubs.obj
 0001:00002b38       __acrt_uninitialize        0000000180003b38 f   MSVCRT:ucrt_stubs.obj
 0001:00002b38       __acrt_uninitialize_critical 0000000180003b38 f   MSVCRT:ucrt_stubs.obj
 0001:00002b38       __scrt_stub_for_acrt_initialize 0000000180003b38 f   MSVCRT:ucrt_stubs.obj
 0001:00002b38       __scrt_stub_for_acrt_thread_attach 0000000180003b38 f   MSVCRT:ucrt_stubs.obj
 0001:00002b38       __scrt_stub_for_acrt_thread_detach 0000000180003b38 f   MSVCRT:ucrt_stubs.obj
 0001:00002b38       __scrt_stub_for_acrt_uninitialize 0000000180003b38 f   MSVCRT:ucrt_stubs.obj
 0001:00002b38       __scrt_stub_for_acrt_uninitialize_critical 0000000180003b38 f   MSVCRT:ucrt_stubs.obj
 0001:00002b38       __vcrt_initialize          0000000180003b38 f   MSVCRT:ucrt_stubs.obj
 0001:00002b38       __vcrt_thread_attach       0000000180003b38 f   MSVCRT:ucrt_stubs.obj
 0001:00002b38       __vcrt_thread_detach       0000000180003b38 f   MSVCRT:ucrt_stubs.obj
 0001:00002b38       __vcrt_uninitialize        0000000180003b38 f   MSVCRT:ucrt_stubs.obj
 0001:00002b38       __vcrt_uninitialize_critical 0000000180003b38 f   MSVCRT:ucrt_stubs.obj
 0001:00002b3c       __scrt_stub_for_is_c_termination_complete 0000000180003b3c f   MSVCRT:ucrt_stubs.obj
 0001:00002b3c       _is_c_termination_complete 0000000180003b3c f   MSVCRT:ucrt_stubs.obj
 0001:00002b50       _guard_dispatch_icall_nop  0000000180003b50 f   MSVCRT:guard_dispatch.obj
 0001:00002b70       _guard_xfg_dispatch_icall_nop 0000000180003b70 f   MSVCRT:guard_xfg_dispatch.obj
 0002:00000000       __imp_RtlCaptureContext    0000000180004000     kernel32:KERNEL32.dll
 0002:00000008       __imp_RtlLookupFunctionEntry 0000000180004008     kernel32:KERNEL32.dll
 0002:00000010       __imp_RtlVirtualUnwind     0000000180004010     kernel32:KERNEL32.dll
 0002:00000018       __imp_UnhandledExceptionFilter 0000000180004018     kernel32:KERNEL32.dll
 0002:00000020       __imp_SetUnhandledExceptionFilter 0000000180004020     kernel32:KERNEL32.dll
 0002:00000028       __imp_GetCurrentProcess    0000000180004028     kernel32:KERNEL32.dll
 0002:00000030       __imp_TerminateProcess     0000000180004030     kernel32:KERNEL32.dll
 0002:00000038       __imp_IsProcessorFeaturePresent 0000000180004038     kernel32:KERNEL32.dll
 0002:00000040       __imp_CloseHandle          0000000180004040     kernel32:KERNEL32.dll
 0002:00000048       __imp_InitializeCriticalSectionAndSpinCount 0000000180004048     kernel32:KERNEL32.dll
 0002:00000050       __imp_DeleteCriticalSection 0000000180004050     kernel32:KERNEL32.dll
 0002:00000058       __imp_CreateEventW         0000000180004058     kernel32:KERNEL32.dll
 0002:00000060       __imp_GetModuleHandleW     0000000180004060     kernel32:KERNEL32.dll
 0002:00000068       __imp_GetProcAddress       0000000180004068     kernel32:KERNEL32.dll
 0002:00000070       __imp_IsDebuggerPresent    0000000180004070     kernel32:KERNEL32.dll
 0002:00000078       __imp_QueryPerformanceCounter 0000000180004078     kernel32:KERNEL32.dll
 0002:00000080       __imp_GetCurrentProcessId  0000000180004080     kernel32:KERNEL32.dll
 0002:00000088       __imp_GetCurrentThreadId   0000000180004088     kernel32:KERNEL32.dll
 0002:00000090       __imp_GetSystemTimeAsFileTime 0000000180004090     kernel32:KERNEL32.dll
 0002:00000098       __imp_DisableThreadLibraryCalls 0000000180004098     kernel32:KERNEL32.dll
 0002:000000a0       __imp_InitializeSListHead  00000001800040a0     kernel32:KERNEL32.dll
 0002:000000a8       \177KERNEL32_NULL_THUNK_DATA 00000001800040a8     kernel32:KERNEL32.dll
 0002:000000b0       __imp_memcpy               00000001800040b0     vcruntime:VCRUNTIME140.dll
 0002:000000b8       __imp_memset               00000001800040b8     vcruntime:VCRUNTIME140.dll
 0002:000000c0       __imp_strchr               00000001800040c0     vcruntime:VCRUNTIME140.dll
 0002:000000c8       __imp___C_specific_handler 00000001800040c8     vcruntime:VCRUNTIME140.dll
 0002:000000d0       __imp___std_type_info_destroy_list 00000001800040d0     vcruntime:VCRUNTIME140.dll
 0002:000000d8       \177VCRUNTIME140_NULL_THUNK_DATA 00000001800040d8     vcruntime:VCRUNTIME140.dll
 0002:000000e0       __imp__errno               00000001800040e0     ucrt:api-ms-win-crt-runtime-l1-1-0.dll
 0002:000000e8       __imp_exit                 00000001800040e8     ucrt:api-ms-win-crt-runtime-l1-1-0.dll
 0002:000000f0       __imp__cexit               00000001800040f0     ucrt:api-ms-win-crt-runtime-l1-1-0.dll
 0002:000000f8       __imp__crt_atexit          00000001800040f8     ucrt:api-ms-win-crt-runtime-l1-1-0.dll
 0002:00000100       __imp__execute_onexit_table 0000000180004100     ucrt:api-ms-win-crt-runtime-l1-1-0.dll
 0002:00000108       __imp__register_onexit_function 0000000180004108     ucrt:api-ms-win-crt-runtime-l1-1-0.dll
 0002:00000110       __imp__initialize_onexit_table 0000000180004110     ucrt:api-ms-win-crt-runtime-l1-1-0.dll
 0002:00000118       __imp__initialize_narrow_environment 0000000180004118     ucrt:api-ms-win-crt-runtime-l1-1-0.dll
 0002:00000120       __imp__configure_narrow_argv 0000000180004120     ucrt:api-ms-win-crt-runtime-l1-1-0.dll
 0002:00000128       __imp__seh_filter_dll      0000000180004128     ucrt:api-ms-win-crt-runtime-l1-1-0.dll
 0002:00000130       __imp__initterm_e          0000000180004130     ucrt:api-ms-win-crt-runtime-l1-1-0.dll
 0002:00000138       __imp__initterm            0000000180004138     ucrt:api-ms-win-crt-runtime-l1-1-0.dll
 0002:00000140       \177api-ms-win-crt-runtime-l1-1-0_NULL_THUNK_DATA 0000000180004140     ucrt:api-ms-win-crt-runtime-l1-1-0.dll
 0002:00000148       __imp___acrt_iob_func      0000000180004148     ucrt:api-ms-win-crt-stdio-l1-1-0.dll
 0002:00000150       __imp_fflush               0000000180004150     ucrt:api-ms-win-crt-stdio-l1-1-0.dll
 0002:00000158       __imp___stdio_common_vsprintf 0000000180004158     ucrt:api-ms-win-crt-stdio-l1-1-0.dll
 0002:00000160       __imp___stdio_common_vfprintf 0000000180004160     ucrt:api-ms-win-crt-stdio-l1-1-0.dll
 0002:00000168       \177api-ms-win-crt-stdio-l1-1-0_NULL_THUNK_DATA 0000000180004168     ucrt:api-ms-win-crt-stdio-l1-1-0.dll
 0002:00000170       __imp_strcmp               0000000180004170     ucrt:api-ms-win-crt-string-l1-1-0.dll
 0002:00000178       __imp__strdup              0000000180004178     ucrt:api-ms-win-crt-string-l1-1-0.dll
 0002:00000178       __imp_strdup               0000000180004178     ucrt:api-ms-win-crt-string-l1-1-0.dll
 0002:00000180       __imp_strlen               0000000180004180     ucrt:api-ms-win-crt-string-l1-1-0.dll
 0002:00000188       __imp_strncpy              0000000180004188     ucrt:api-ms-win-crt-string-l1-1-0.dll
 0002:00000190       \177api-ms-win-crt-string-l1-1-0_NULL_THUNK_DATA 0000000180004190     ucrt:api-ms-win-crt-string-l1-1-0.dll
 0002:00000198       __guard_check_icall_fptr   0000000180004198     MSVCRT:guard_support.obj
 0002:000001a0       __guard_xfg_check_icall_fptr 00000001800041a0     MSVCRT:guard_support.obj
 0002:000001a8       __guard_dispatch_icall_fptr 00000001800041a8     MSVCRT:guard_support.obj
 0002:000001b0       __guard_xfg_dispatch_icall_fptr 00000001800041b0     MSVCRT:guard_support.obj
 0002:000001b8       __guard_xfg_table_dispatch_icall_fptr 00000001800041b8     MSVCRT:guard_support.obj
 0002:000001c0       __castguard_check_failure_os_handled_fptr 00000001800041c0     MSVCRT:guard_support.obj
 0002:000001c8       __guard_memcpy_fptr        00000001800041c8     vcruntime:softmemtag.obj
 0002:000001d0       __xc_a                     00000001800041d0     MSVCRT:initializers.obj
 0002:000001d8       __xc_z                     00000001800041d8     MSVCRT:initializers.obj
 0002:000001e0       __xi_a                     00000001800041e0     MSVCRT:initializers.obj
 0002:000001f0       __xi_z                     00000001800041f0     MSVCRT:initializers.obj
 0002:000001f8       __xl_a                     00000001800041f8     MSVCRT:tlssup.obj
 0002:00000200       __xl_z                     0000000180004200     MSVCRT:tlssup.obj
 0002:00000208       __xp_a                     0000000180004208     MSVCRT:initializers.obj
 0002:00000210       __xp_z                     0000000180004210     MSVCRT:initializers.obj
 0002:00000218       __xt_a                     0000000180004218     MSVCRT:initializers.obj
 0002:00000220       __xt_z                     0000000180004220     MSVCRT:initializers.obj
 0002:00000230       g_refKindStr               0000000180004230     libgetfldecl004.obj
 0002:000003e0       ??_C@_09BPLDFGCI@unknown_0@ 00000001800043e0     libgetfldecl004.obj
 0002:000003f0       ??_C@_0BL@FPNMECJD@JVMTI_HEAP_REFERENCE_CLASS@ 00000001800043f0     libgetfldecl004.obj
 0002:00000410       ??_C@_0BL@FKGKKLNM@JVMTI_HEAP_REFERENCE_FIELD@ 0000000180004410     libgetfldecl004.obj
 0002:00000430       ??_C@_0CD@CAEHCFJF@JVMTI_HEAP_REFERENCE_ARRAY_ELEM@ 0000000180004430     libgetfldecl004.obj
 0002:00000458       ??_C@_0CC@DNEBMCNK@JVMTI_HEAP_REFERENCE_CLASS_LOAD@ 0000000180004458     libgetfldecl004.obj
 0002:00000480       ??_C@_0BN@CJMIPEBB@JVMTI_HEAP_REFERENCE_SIGNERS@ 0000000180004480     libgetfldecl004.obj
 0002:000004a0       ??_C@_0CH@HBOIDPEB@JVMTI_HEAP_REFERENCE_PROTECTION@ 00000001800044a0     libgetfldecl004.obj
 0002:000004c8       ??_C@_0BP@MDKGDGKL@JVMTI_HEAP_REFERENCE_INTERFACE@ 00000001800044c8     libgetfldecl004.obj
 0002:000004e8       ??_C@_0CC@JJMIHNJH@JVMTI_HEAP_REFERENCE_STATIC_FIE@ 00000001800044e8     libgetfldecl004.obj
 0002:00000510       ??_C@_0CD@IDHEEGID@JVMTI_HEAP_REFERENCE_CONSTANT_P@ 0000000180004510     libgetfldecl004.obj
 0002:00000538       ??_C@_0CA@EFFCHNG@JVMTI_HEAP_REFERENCE_SUPERCLASS@ 0000000180004538     libgetfldecl004.obj
 0002:00000558       ??_C@_0L@PCDFHGCJ@unknown_11@ 0000000180004558     libgetfldecl004.obj
 0002:00000568       ??_C@_0L@NJBICFOK@unknown_12@ 0000000180004568     libgetfldecl004.obj
 0002:00000578       ??_C@_0L@MAADBEKL@unknown_13@ 0000000180004578     libgetfldecl004.obj
 0002:00000588       ??_C@_0L@IPECICGM@unknown_14@ 0000000180004588     libgetfldecl004.obj
 0002:00000598       ??_C@_0L@JGFJLDCN@unknown_15@ 0000000180004598     libgetfldecl004.obj
 0002:000005a8       ??_C@_0L@LNHEOAOO@unknown_16@ 00000001800045a8     libgetfldecl004.obj
 0002:000005b8       ??_C@_0L@KEGPNBKP@unknown_17@ 00000001800045b8     libgetfldecl004.obj
 0002:000005c8       ??_C@_0L@CDPHMNGA@unknown_18@ 00000001800045c8     libgetfldecl004.obj
 0002:000005d8       ??_C@_0L@DKOMPMCB@unknown_19@ 00000001800045d8     libgetfldecl004.obj
 0002:000005e8       ??_C@_0L@OJGIPJDB@unknown_20@ 00000001800045e8     libgetfldecl004.obj
 0002:000005f8       ??_C@_0CA@KAOFNDEM@JVMTI_HEAP_REFERENCE_JNI_GLOBAL@ 00000001800045f8     libgetfldecl004.obj
 0002:00000618       ??_C@_0CC@HPFAJBK@JVMTI_HEAP_REFERENCE_SYSTEM_CLA@ 0000000180004618     libgetfldecl004.obj
 0002:00000640       ??_C@_0BN@FDEGFOHC@JVMTI_HEAP_REFERENCE_MONITOR@ 0000000180004640     libgetfldecl004.obj
 0002:00000660       ??_C@_0CB@HKIBCMAJ@JVMTI_HEAP_REFERENCE_STACK_LOCA@ 0000000180004660     libgetfldecl004.obj
 0002:00000688       ??_C@_0BP@EAACMMOE@JVMTI_HEAP_REFERENCE_JNI_LOCAL@ 0000000180004688     libgetfldecl004.obj
 0002:000006a8       ??_C@_0BM@IJDEOGOE@JVMTI_HEAP_REFERENCE_THREAD@ 00000001800046a8     libgetfldecl004.obj
 0002:000006c8       ??_C@_0BL@EDGPPKC@JVMTI_HEAP_REFERENCE_OTHER@ 00000001800046c8     libgetfldecl004.obj
 0002:000006e4       ??_C@_04BCJPDBDA@Code@     00000001800046e4     libgetfldecl004.obj
 0002:000006f0       ??_C@_0BA@OCLMCFKC@LineNumberTable@ 00000001800046f0     libgetfldecl004.obj
 0002:00000700       ??_C@_0BD@CPAEPILC@LocalVariableTable@ 0000000180004700     libgetfldecl004.obj
 0002:00000718       ??_C@_0BH@NMBDNHBD@LocalVariableTypeTable@ 0000000180004718     libgetfldecl004.obj
 0002:00000730       ??_C@_0O@HIHEEDNJ@StackMapTable@ 0000000180004730     libgetfldecl004.obj
 0002:00000740       ??_C@_0BA@CHLCEAPH@staticField_ii1@ 0000000180004740     libgetfldecl004.obj
 0002:00000750       ??_C@_01JPJNBJEM@I@        0000000180004750     libgetfldecl004.obj
 0002:00000758       ??_C@_0BA@MJPBDDE@staticField_ii2@ 0000000180004758     libgetfldecl004.obj
 0002:00000768       ??_C@_0BA@CKCFMFCB@staticField_ic1@ 0000000180004768     libgetfldecl004.obj
 0002:00000778       ??_C@_0BC@FGNMMC@instanceField_ic1@ 0000000180004778     libgetfldecl004.obj
 0002:00000790       ??_C@_0BA@BAIJGOC@staticField_ic2@ 0000000180004790     libgetfldecl004.obj
 0002:000007a0       ??_C@_0BC@CLHLIPAB@instanceField_ic2@ 00000001800047a0     libgetfldecl004.obj
 0002:000007b8       ??_C@_0BA@CNJBPCL@staticField_oi1@ 00000001800047b8     libgetfldecl004.obj
 0002:000007c8       ??_C@_0BA@CJPEEMOI@staticField_oi2@ 00000001800047c8     libgetfldecl004.obj
 0002:000007d8       ??_C@_0BA@PEOJKPN@staticField_oc1@ 00000001800047d8     libgetfldecl004.obj
 0002:000007e8       ??_C@_0BC@CFDNIDBO@instanceField_oc1@ 00000001800047e8     libgetfldecl004.obj
 0002:00000800       ??_C@_0BA@CEGDMJDO@staticField_oc2@ 0000000180004800     libgetfldecl004.obj
 0002:00000810       ??_C@_0BC@OBANANN@instanceField_oc2@ 0000000180004810     libgetfldecl004.obj
 0002:00000828       ??_C@_0L@HCDIAMJG@?9?5?$CFs?0?5?$CFd?3?5@ 0000000180004828     libgetfldecl004.obj
 0002:00000840       ??_C@_0JI@HLPECLFI@?$CD?5?4?4?4?6?$CD?5ERROR?3?5too?5many?5complai@ 0000000180004840     libgetfldecl004.obj
 0002:000008e0       ??_C@_0ED@JNEKCCOB@The?5following?5fake?5exception?5st@ 00000001800048e0     libgetfldecl004.obj
 0002:00000928       ??_C@_0CN@FCNMDFBH@nsk?4share?4Fake_Exception_for_RU@ 0000000180004928     libgetfldecl004.obj
 0002:00000958       ??_C@_08PGFFNAEI@?$CI?$CFs?3?$CFd?$CJ?5@ 0000000180004958     libgetfldecl004.obj
 0002:00000968       ??_C@_0DP@IENMAEGI@s?2test?2hotspot?2jtreg?2vmTestbase@ 0000000180004968     libgetfldecl004.obj
 0002:000009a8       ??_C@_0BL@NDJLFFJB@?7at?5nsk_lvcomplain?$CI?$CFs?3?$CFd?$CJ?6@ 00000001800049a8     libgetfldecl004.obj
 0002:000009c8       ??_C@_0BC@JOOKAFKF@?$CD?5ERROR?3?5?$CFs?0?5?$CFd?3?5@ 00000001800049c8     libgetfldecl004.obj
 0002:000009e0       ??_C@_09KJEAHMEH@?$CD?5ERROR?3?5@ 00000001800049e0     libgetfldecl004.obj
 0002:000009ec       ??_C@_02GPIOPFAK@?$DO?$DO@ 00000001800049ec     libgetfldecl004.obj
 0002:000009f0       ??_C@_02FODMEDOG@?$DM?$DM@ 00000001800049f0     libgetfldecl004.obj
 0002:000009f4       ??_C@_02DJGKEECL@?4?4@     00000001800049f4     libgetfldecl004.obj
 0002:000009f8       ??_C@_0O@CJPGJOAF@?9?5?$CFs?0?5?$CFd?3?5?$CFs?5@ 00000001800049f8     libgetfldecl004.obj
 0002:00000a08       ??_C@_0CB@IAKPDOIC@?$CD?5?5?5verified?5assertion?5is?5FALSE@ 0000000180004a08     libgetfldecl004.obj
 0002:00000a30       ??_C@_0CO@LGONDEPD@stdout?3?5fflush?5failed?5?9?5err?$DN?$CFd?5@ 0000000180004a30     libgetfldecl004.obj
 0002:00000a60       ??_C@_0CO@KBGKJPBD@stderr?3?5fflush?5failed?5?9?5err?$DN?$CFd?5@ 0000000180004a60     libgetfldecl004.obj
 0002:00000a90       ??_C@_0BB@JCNMKLLK@JVMTI_ERROR_NONE@ 0000000180004a90     libgetfldecl004.obj
 0002:00000aa8       ??_C@_0BL@LDIMKLPH@JVMTI_ERROR_INVALID_THREAD@ 0000000180004aa8     libgetfldecl004.obj
 0002:00000ac8       ??_C@_0CB@PJFPAIKJ@JVMTI_ERROR_INVALID_THREAD_GROU@ 0000000180004ac8     libgetfldecl004.obj
 0002:00000af0       ??_C@_0BN@LLMKHMNF@JVMTI_ERROR_INVALID_PRIORITY@ 0000000180004af0     libgetfldecl004.obj
 0002:00000b10       ??_C@_0CB@MBOFKAGB@JVMTI_ERROR_THREAD_NOT_SUSPENDE@ 0000000180004b10     libgetfldecl004.obj
 0002:00000b38       ??_C@_0BN@FABOLPBI@JVMTI_ERROR_THREAD_SUSPENDED@ 0000000180004b38     libgetfldecl004.obj
 0002:00000b58       ??_C@_0BN@FDGNOBJM@JVMTI_ERROR_THREAD_NOT_ALIVE@ 0000000180004b58     libgetfldecl004.obj
 0002:00000b78       ??_C@_0BL@GOBIFKNJ@JVMTI_ERROR_INVALID_OBJECT@ 0000000180004b78     libgetfldecl004.obj
 0002:00000b98       ??_C@_0BK@FCMAJPPC@JVMTI_ERROR_INVALID_CLASS@ 0000000180004b98     libgetfldecl004.obj
 0002:00000bb8       ??_C@_0BP@IKLLBKEB@JVMTI_ERROR_CLASS_NOT_PREPARED@ 0000000180004bb8     libgetfldecl004.obj
 0002:00000bd8       ??_C@_0BN@KLPPLKG@JVMTI_ERROR_INVALID_METHODID@ 0000000180004bd8     libgetfldecl004.obj
 0002:00000bf8       ??_C@_0BN@BCEKOKND@JVMTI_ERROR_INVALID_LOCATION@ 0000000180004bf8     libgetfldecl004.obj
 0002:00000c18       ??_C@_0BM@DFDGPME@JVMTI_ERROR_INVALID_FIELDID@ 0000000180004c18     libgetfldecl004.obj
 0002:00000c38       ??_C@_0BL@NELIEPEC@JVMTI_ERROR_NO_MORE_FRAMES@ 0000000180004c38     libgetfldecl004.obj
 0002:00000c58       ??_C@_0BJ@BDBECFDM@JVMTI_ERROR_OPAQUE_FRAME@ 0000000180004c58     libgetfldecl004.obj
 0002:00000c78       ??_C@_0BK@MIIFNLOB@JVMTI_ERROR_TYPE_MISMATCH@ 0000000180004c78     libgetfldecl004.obj
 0002:00000c98       ??_C@_0BJ@HPCAOILC@JVMTI_ERROR_INVALID_SLOT@ 0000000180004c98     libgetfldecl004.obj
 0002:00000cb8       ??_C@_0BG@CHILOPNI@JVMTI_ERROR_DUPLICATE@ 0000000180004cb8     libgetfldecl004.obj
 0002:00000cd0       ??_C@_0BG@DIEMLHKM@JVMTI_ERROR_NOT_FOUND@ 0000000180004cd0     libgetfldecl004.obj
 0002:00000ce8       ??_C@_0BM@NHMCKHOB@JVMTI_ERROR_INVALID_MONITOR@ 0000000180004ce8     libgetfldecl004.obj
 0002:00000d08       ??_C@_0BO@PPEDAJGL@JVMTI_ERROR_NOT_MONITOR_OWNER@ 0000000180004d08     libgetfldecl004.obj
 0002:00000d28       ??_C@_0BG@FCAIPEID@JVMTI_ERROR_INTERRUPT@ 0000000180004d28     libgetfldecl004.obj
 0002:00000d40       ??_C@_0CB@EGDBNKOI@JVMTI_ERROR_INVALID_CLASS_FORMA@ 0000000180004d40     libgetfldecl004.obj
 0002:00000d68       ??_C@_0CG@DGKOGIAL@JVMTI_ERROR_CIRCULAR_CLASS_DEFI@ 0000000180004d68     libgetfldecl004.obj
 0002:00000d90       ??_C@_0BP@ICEALPKC@JVMTI_ERROR_FAILS_VERIFICATION@ 0000000180004d90     libgetfldecl004.obj
 0002:00000db0       ??_C@_0DC@JDACLMIO@JVMTI_ERROR_UNSUPPORTED_REDEFIN@ 0000000180004db0     libgetfldecl004.obj
 0002:00000de8       ??_C@_0DE@GKDKNOMJ@JVMTI_ERROR_UNSUPPORTED_REDEFIN@ 0000000180004de8     libgetfldecl004.obj
 0002:00000e20       ??_C@_0BO@LAFKIOG@JVMTI_ERROR_INVALID_TYPESTATE@ 0000000180004e20     libgetfldecl004.obj
 0002:00000e40       ??_C@_0DH@INDGCLLB@JVMTI_ERROR_UNSUPPORTED_REDEFIN@ 0000000180004e40     libgetfldecl004.obj
 0002:00000e78       ??_C@_0DE@NHEOMMGI@JVMTI_ERROR_UNSUPPORTED_REDEFIN@ 0000000180004e78     libgetfldecl004.obj
 0002:00000eb0       ??_C@_0CA@EKPNJOEP@JVMTI_ERROR_UNSUPPORTED_VERSION@ 0000000180004eb0     libgetfldecl004.obj
 0002:00000ed0       ??_C@_0BN@OFFMAHHL@JVMTI_ERROR_NAMES_DONT_MATCH@ 0000000180004ed0     libgetfldecl004.obj
 0002:00000ef0       ??_C@_0DN@HHBBLAKE@JVMTI_ERROR_UNSUPPORTED_REDEFIN@ 0000000180004ef0     libgetfldecl004.obj
 0002:00000f30       ??_C@_0DO@HMBGBGNA@JVMTI_ERROR_UNSUPPORTED_REDEFIN@ 0000000180004f30     libgetfldecl004.obj
 0002:00000f70       ??_C@_0BP@PBECGKHJ@JVMTI_ERROR_UNMODIFIABLE_CLASS@ 0000000180004f70     libgetfldecl004.obj
 0002:00000f90       ??_C@_0BK@CANILEHF@JVMTI_ERROR_NOT_AVAILABLE@ 0000000180004f90     libgetfldecl004.obj
 0002:00000fb0       ??_C@_0CE@INJKMEFK@JVMTI_ERROR_MUST_POSSESS_CAPABI@ 0000000180004fb0     libgetfldecl004.obj
 0002:00000fd8       ??_C@_0BJ@LBFPFPDM@JVMTI_ERROR_NULL_POINTER@ 0000000180004fd8     libgetfldecl004.obj
 0002:00000ff8       ??_C@_0BP@CHJPNNEM@JVMTI_ERROR_ABSENT_INFORMATION@ 0000000180004ff8     libgetfldecl004.obj
 0002:00001018       ??_C@_0BP@OMFMNLC@JVMTI_ERROR_INVALID_EVENT_TYPE@ 0000000180005018     libgetfldecl004.obj
 0002:00001038       ??_C@_0BN@BIBNPHHO@JVMTI_ERROR_ILLEGAL_ARGUMENT@ 0000000180005038     libgetfldecl004.obj
 0002:00001058       ??_C@_0BK@KKNDHDCE@JVMTI_ERROR_NATIVE_METHOD@ 0000000180005058     libgetfldecl004.obj
 0002:00001078       ??_C@_0BK@PMKCFHAE@JVMTI_ERROR_OUT_OF_MEMORY@ 0000000180005078     libgetfldecl004.obj
 0002:00001098       ??_C@_0BK@NNJBDMNB@JVMTI_ERROR_ACCESS_DENIED@ 0000000180005098     libgetfldecl004.obj
 0002:000010b8       ??_C@_0BI@GHECLMNC@JVMTI_ERROR_WRONG_PHASE@ 00000001800050b8     libgetfldecl004.obj
 0002:000010d0       ??_C@_0BF@OLIHJOII@JVMTI_ERROR_INTERNAL@ 00000001800050d0     libgetfldecl004.obj
 0002:000010e8       ??_C@_0BO@EOHGKJHI@JVMTI_ERROR_UNATTACHED_THREAD@ 00000001800050e8     libgetfldecl004.obj
 0002:00001108       ??_C@_0CA@LKHFDACL@JVMTI_ERROR_INVALID_ENVIRONMENT@ 0000000180005108     libgetfldecl004.obj
 0002:00001128       ??_C@_0BA@MMFHLOKK@?$DMunknown?5error?$DO@ 0000000180005128     libgetfldecl004.obj
 0002:00001138       ??_C@_0CF@CBHOKDB@throwable?5?$DN?5jni?9?$DOExceptionOccur@ 0000000180005138     libgetfldecl004.obj
 0002:00001160       ??_C@_03OFAPEBGM@?$CFs?6@  0000000180005160     libgetfldecl004.obj
 0002:00001168       ??_C@_0DM@LPIGEGNJ@s?2test?2hotspot?2jtreg?2vmTestbase@ 0000000180005168     libgetfldecl004.obj
 0002:000011a8       ??_C@_0CC@NFCNPEPK@Exception?5in?5JNI?5call?5?$CIcleared?$CJ@ 00000001800051a8     libgetfldecl004.obj
 0002:000011d0       ??_C@_0BJ@IBAKFIKF@jni?9?$DOExceptionDescribe?$CI?$CJ@ 00000001800051d0     libgetfldecl004.obj
 0002:000011f0       ??_C@_0BG@GGKALKMH@jni?9?$DOExceptionClear?$CI?$CJ@ 00000001800051f0     libgetfldecl004.obj
 0002:00001208       ??_C@_0CF@JMGFGJLJ@?$CD?5?5?5verified?5JNI?5assertion?5is?5F@ 0000000180005208     libgetfldecl004.obj
 0002:00001230       ??_C@_0CB@MLNJNCLJ@?5?5jvmti?5error?3?5code?$DN?$CFd?0?5name?$DN?$CFs@ 0000000180005230     libgetfldecl004.obj
 0002:00001258       ??_C@_0CD@OHBGDKMK@?$CD?5?5?5jvmti?5error?3?5code?$DN?$CFd?0?5name?$DN@ 0000000180005258     libgetfldecl004.obj
 0002:00001280       ??_C@_0CG@JNNCGPHB@?$CD?5?5?5error?5expected?3?5code?$DN?$CFd?0?5na@ 0000000180005280     libgetfldecl004.obj
 0002:000012b0       ??_C@_0EB@IMGKPCGE@?$CIstr_obj?5?$DN?5jni?9?$DONewStringUTF?$CIco@ 00000001800052b0     libgetfldecl004.obj
 0002:00001300       ??_C@_0EA@HFOGGBCC@s?2test?2hotspot?2jtreg?2vmTestbase@ 0000000180005300     libgetfldecl004.obj
 0002:00001340       ??_C@_05KKCIMGE@error@     0000000180005340     libgetfldecl004.obj
 0002:00001348       ??_C@_0CJ@JACLEAA@Test?5failed?5by?5setFailStatus?$CI?$CJ?4@ 0000000180005348     libgetfldecl004.obj
 0002:00001380       ??_C@_0EA@PNBCDMOA@s?2test?2hotspot?2jtreg?2vmTestbase@ 0000000180005380     libgetfldecl004.obj
 0002:000013c0       ??_C@_0DI@ILAHDLMP@?$CI?$CKagentThreadProc?$CJ?$CIjvmti_env?0?5a@ 00000001800053c0     libgetfldecl004.obj
 0002:000013f8       ??_C@_0BD@KDBALNLB@JVMTI?5agent?5thread@ 00000001800053f8     libgetfldecl004.obj
 0002:00001410       ??_C@_0BB@NOKBFPFO@java?1lang?1Thread@ 0000000180005410     libgetfldecl004.obj
 0002:00001424       ??_C@_06FALKBLGB@?$DMinit?$DO@ 0000000180005424     libgetfldecl004.obj
 0002:00001430       ??_C@_0BG@IKDDPPGD@?$CILjava?1lang?1String?$DL?$CJV@ 0000000180005430     libgetfldecl004.obj
 0002:00001450       ??_C@_0EB@IFJBFEKC@?$CIthreadClass?5?$DN?5jni_env?9?$DOFindCla@ 0000000180005450     libgetfldecl004.obj
 0002:000014a0       ??_C@_0GF@FGFIBKKL@?$CIthreadCtor?5?$DN?5jni_env?9?$DOGetMetho@ 00000001800054a0     libgetfldecl004.obj
 0002:00001508       ??_C@_0DN@NCPDJLOG@?$CIthreadName?5?$DN?5jni_env?9?$DONewStrin@ 0000000180005508     libgetfldecl004.obj
 0002:00001550       ??_C@_0FE@PFKODBGC@?$CIthreadObject?5?$DN?5jni_env?9?$DONewObj@ 0000000180005550     libgetfldecl004.obj
 0002:000015b0       ??_C@_0ED@HOBAHHJI@?$CIthreadGlobalRef?5?$DN?5jni_env?9?$DONew@ 00000001800055b0     libgetfldecl004.obj
 0002:00001600       ??_C@_0FN@HNJJAHFC@jvmti_env?9?$DORunAgentThread?$CIagent@ 0000000180005600     libgetfldecl004.obj
 0002:00001660       ??_C@_0EA@MOJDNKDF@Debuggee?5status?5sync?5aborted?5be@ 0000000180005660     libgetfldecl004.obj
 0002:000016a0       ??_C@_0EA@EEOEJAEN@status?5?$DN?5syncDebuggeeStatus?$CIjni@ 00000001800056a0     libgetfldecl004.obj
 0002:000016e0       ??_C@_0BL@JBCFNBMB@nsk_jvmti_resetAgentData?$CI?$CJ@ 00000001800056e0     libgetfldecl004.obj
 0002:00001700       ??_C@_0EL@LPBEELIP@s?2test?2hotspot?2jtreg?2vmTestbase@ 0000000180005700     libgetfldecl004.obj
 0002:00001750       ??_C@_0CK@JDAMFDMJ@jvmti?9?$DOSetTag?$CIo?0?5tag?$CJ?5?$DN?$DN?5JVMTI_@ 0000000180005750     libgetfldecl004.obj
 0002:00001780       ??_C@_0CC@DAMNHKNI@Can?8t?5set?5tag?5?$CFli?5for?5object?5?$CFl@ 0000000180005780     libgetfldecl004.obj
 0002:000017a8       ??_C@_0DL@HAJPNKEF@jvmti?9?$DOGetObjectHashCode?$CIo?0?5?$CGha@ 00000001800057a8     libgetfldecl004.obj
 0002:000017e8       ??_C@_0BL@JFPIEOBF@Can?8t?5get?5hash?5object?5?$CFlx?6@ 00000001800057e8     libgetfldecl004.obj
 0002:00001808       ??_C@_0BG@DICPHBKN@setTag?3?5?$CF08x?5?$DM?9?5?$CF?53li@ 0000000180005808     libgetfldecl004.obj
 0002:00001820       ??_C@_0DH@FCEEBDMJ@?$CIs?5?$DN?5jni?9?$DOGetStringUTFChars?$CIsIn@ 0000000180005820     libgetfldecl004.obj
 0002:00001858       ??_C@_0BJ@OKKGHDCN@Can?8t?5get?5string?5at?5?$CF?$CDp?6@ 0000000180005858     libgetfldecl004.obj
 0002:00001878       ??_C@_0BP@EKFLGGFJ@Can?8t?5get?5string?5at?5?$CF?$CDp?3?5null?6@ 0000000180005878     libgetfldecl004.obj
 0002:00001898       ??_C@_06ICODBHCL@?5?1?1?5?$CFs@ 0000000180005898     libgetfldecl004.obj
 0002:000018a0       ??_C@_0DB@KGFPLEGO@?$CIr?5?$DN?5jvmti?9?$DOGetTag?$CIo?0?5?$CGtag?$CJ?$CJ?5?$DN?$DN@ 00000001800058a0     libgetfldecl004.obj
 0002:000018d8       ??_C@_0CO@PDAGBCGJ@Can?8t?5GetTag?5for?5object?5?$CFlx?4?5Re@ 00000001800058d8     libgetfldecl004.obj
 0002:00001908       ??_C@_0CH@HPEODOHC@TEST_BUG?3?5Max?4?5number?5of?5refs?5r@ 0000000180005908     libgetfldecl004.obj
 0002:00001930       ??_C@_0DI@PHFCABIM@?$CIr?5?$DN?5jvmti?9?$DOGetTag?$CIfrom?0?5?$CGtagFr@ 0000000180005930     libgetfldecl004.obj
 0002:00001968       ??_C@_0DI@MDEGFNKD@TEST_BUG?3?5Can?8t?5GetTag?5for?5obje@ 0000000180005968     libgetfldecl004.obj
 0002:000019a0       ??_C@_0DE@MLELJAHM@?$CIr?5?$DN?5jvmti?9?$DOGetTag?$CIto?0?5?$CGtagTo?$CJ?$CJ@ 00000001800059a0     libgetfldecl004.obj
 0002:000019d8       ??_C@_09OPJEJKBL@printdump@ 00000001800059d8     libgetfldecl004.obj
 0002:000019e8       ??_C@_0CJ@KCDEKOCJ@Wrong?5result?5of?5a?5valid?5call?5to@ 00000001800059e8     libgetfldecl004.obj
 0002:00001a18       ??_C@_0CH@CDOJMNAO@JVMTI?5client?5was?5not?5properly?5l@ 0000000180005a18     libgetfldecl004.obj
 0002:00001a40       ??_C@_0CG@BCDHGIMH@?$CI?$CFd?$CJ?5cannot?5get?5field?5ID?5for?5?$CFs@ 0000000180005a40     libgetfldecl004.obj
 0002:00001a68       ??_C@_0DH@ODMPGCPO@?$CIGetFieldDeclaringClass?$CD?$CFd?$CJ?5une@ 0000000180005a68     libgetfldecl004.obj
 0002:00001aa0       ??_C@_0DC@CKFFJKGO@?$CIGetClassSignature?$CD?$CFd?$CJ?5unexpect@ 0000000180005aa0     libgetfldecl004.obj
 0002:00001ad8       ??_C@_0BE@CKCLPLAD@?$DO?$DO?$DO?5?$CFd?5?9?9?5?$CFs?3?5?$CC?$CFs?$CC?6@ 0000000180005ad8     libgetfldecl004.obj
 0002:00001af0       ??_C@_0CE@BHBHGAK@?$CI?$CFd?$CJ?5unexpected?5declaringClass?3@ 0000000180005af0     libgetfldecl004.obj
 0002:00001b30       ??_C@_1EC@JIJBPKFM@?$AAa?$AAp?$AAi?$AA?9?$AAm?$AAs?$AA?9?$AAw?$AAi?$AAn?$AA?9?$AAc?$AAo?$AAr?$AAe@ 0000000180005b30     MSVCRT:thread_safe_statics.obj
 0002:00001b78       ??_C@_1BK@MGMFAEKH@?$AAk?$AAe?$AAr?$AAn?$AAe?$AAl?$AA3?$AA2?$AA?4?$AAd?$AAl?$AAl@ 0000000180005b78     MSVCRT:thread_safe_statics.obj
 0002:00001b98       ??_C@_0BJ@JEBJOJFJ@SleepConditionVariableCS@ 0000000180005b98     MSVCRT:thread_safe_statics.obj
 0002:00001bb8       ??_C@_0BJ@PGPPEPCC@WakeAllConditionVariable@ 0000000180005bb8     MSVCRT:thread_safe_statics.obj
 0002:00001bd8       _pDefaultRawDllMain        0000000180005bd8     MSVCRT:dll_dllmain.obj
 0002:00001bd8       _pRawDllMain               0000000180005bd8     MSVCRT:dll_dllmain.obj
 0002:00001be0       __xmm@ffffffffffffffffffffffffffffffff 0000000180005be0     MSVCRT:utility.obj
 0002:00001bf0       _load_config_used          0000000180005bf0     MSVCRT:loadcfg.obj
 0002:00001e00       _tls_used                  0000000180005e00     MSVCRT:tlssup.obj
 0002:00001e28       __volatile_metadata        0000000180005e28     <linker-defined>
 0002:000021e8       __rtc_iaa                  00000001800061e8     MSVCRT:initsect.obj
 0002:000021f0       __rtc_izz                  00000001800061f0     MSVCRT:initsect.obj
 0002:000021f8       __rtc_taa                  00000001800061f8     MSVCRT:initsect.obj
 0002:00002200       __rtc_tzz                  0000000180006200     MSVCRT:initsect.obj
 0002:00002208       _tls_start                 0000000180006208     MSVCRT:tlssup.obj
 0002:0000220c       _Init_thread_epoch         000000018000620c     MSVCRT:thread_safe_statics.obj
 0002:00002210       _tls_end                   0000000180006210     MSVCRT:tlssup.obj
 0002:000028ec       __IMPORT_DESCRIPTOR_KERNEL32 00000001800068ec     kernel32:KERNEL32.dll
 0002:00002900       __IMPORT_DESCRIPTOR_VCRUNTIME140 0000000180006900     vcruntime:VCRUNTIME140.dll
 0002:00002914       __IMPORT_DESCRIPTOR_api-ms-win-crt-runtime-l1-1-0 0000000180006914     ucrt:api-ms-win-crt-runtime-l1-1-0.dll
 0002:00002928       __IMPORT_DESCRIPTOR_api-ms-win-crt-stdio-l1-1-0 0000000180006928     ucrt:api-ms-win-crt-stdio-l1-1-0.dll
 0002:0000293c       __IMPORT_DESCRIPTOR_api-ms-win-crt-string-l1-1-0 000000018000693c     ucrt:api-ms-win-crt-string-l1-1-0.dll
 0002:00002950       __NULL_IMPORT_DESCRIPTOR   0000000180006950     kernel32:KERNEL32.dll
 0003:00000150       _Init_global_epoch         0000000180007150     MSVCRT:thread_safe_statics.obj
 0003:00000160       __security_cookie          0000000180007160     MSVCRT:gs_cookie.obj
 0003:00000168       __security_cookie_complement 0000000180007168     MSVCRT:gs_cookie.obj
 0003:00000170       __scrt_native_dllmain_reason 0000000180007170     MSVCRT:utility.obj
 0003:00000178       __isa_available            0000000180007178     MSVCRT:cpu_disp.obj
 0003:0000017c       __isa_enabled              000000018000717c     MSVCRT:cpu_disp.obj
 0003:00000180       __memset_fast_string_threshold 0000000180007180     MSVCRT:cpu_disp.obj
 0003:00000188       __memset_nt_threshold      0000000180007188     MSVCRT:cpu_disp.obj
 0003:00000190       __scrt_ucrt_dll_is_in_use  0000000180007190     MSVCRT:ucrt_stubs.obj
 0003:000001a0       g_wrongHeapCallbacks       00000001800071a0     libgetfldecl004.obj
 0003:00000220       g_szTagInfo                0000000180007220     libgetfldecl004.obj
 0003:00002160       g_tagFlags                 0000000180009160     libgetfldecl004.obj
 0003:00002548       g_refsToVerifyCnt          0000000180009548     libgetfldecl004.obj
 0003:0000254c       g_fakeUserData             000000018000954c     libgetfldecl004.obj
 0003:00002550       g_tagVisitCount            0000000180009550     libgetfldecl004.obj
 0003:000034f0       g_refsToVerify             000000018000a4f0     libgetfldecl004.obj
 0003:0001abf0       g_userDataError            0000000180021bf0     libgetfldecl004.obj
 0003:0001ad90       ?_OptionsStorage@?1??__local_stdio_printf_options@@9@4_KA 0000000180021d90     libgetfldecl004.obj
 0003:0001b358       _tls_index                 0000000180022358     MSVCRT:tlssup.obj
 0003:0001b360       __scrt_current_native_startup_state 0000000180022360     MSVCRT:utility.obj
 0003:0001b368       __scrt_native_startup_lock 0000000180022368     MSVCRT:utility.obj
 0003:0001b3a8       __scrt_debugger_hook_flag  00000001800223a8     MSVCRT:utility_desktop.obj
 0003:0001b3b0       ?__type_info_root_node@@3U__type_info_node@@A 00000001800223b0     MSVCRT:tncleanup.obj
 0003:0001b3c0       ?_OptionsStorage@?1??__local_stdio_scanf_options@@9@4_KA 00000001800223c0     MSVCRT:default_local_stdio_options.obj
 0003:0001b3c8       __favor                    00000001800223c8     MSVCRT:cpu_disp.obj
 0003:0001b3d0       __dyn_tls_init_callback    00000001800223d0     <common>

 entry point at        0001:00002260

 Static symbols

 0000:fffdb000       .debug$S                   0000000180000000     getfldecl004.exp
 0000:fffdb000       .debug$S                   0000000180000000     vcruntime:VCRUNTIME140.dll
 0000:fffdb000       .debug$S                   0000000180000000     vcruntime:VCRUNTIME140.dll
 0000:fffdb000       .debug$S                   0000000180000000     vcruntime:VCRUNTIME140.dll
 0000:fffdb000       .debug$S                   0000000180000000     vcruntime:VCRUNTIME140.dll
 0000:fffdb000       .debug$S                   0000000180000000     vcruntime:VCRUNTIME140.dll
 0000:fffdb000       .debug$S                   0000000180000000     vcruntime:VCRUNTIME140.dll
 0000:fffdb000       .debug$S                   0000000180000000     vcruntime:VCRUNTIME140.dll
 0000:fffdb000       .debug$S                   0000000180000000     ucrt:api-ms-win-crt-convert-l1-1-0.dll
 0002:ffffc000       .idata$6                   0000000180000000     ucrt:api-ms-win-crt-convert-l1-1-0.dll
 0000:fffdb000       .debug$S                   0000000180000000     ucrt:api-ms-win-crt-heap-l1-1-0.dll
 0000:fffdb000       .debug$S                   0000000180000000     ucrt:api-ms-win-crt-heap-l1-1-0.dll
 0000:fffdb000       .debug$S                   0000000180000000     ucrt:api-ms-win-crt-heap-l1-1-0.dll
 0000:fffdb000       .debug$S                   0000000180000000     ucrt:api-ms-win-crt-heap-l1-1-0.dll
 0002:ffffc000       .idata$6                   0000000180000000     ucrt:api-ms-win-crt-heap-l1-1-0.dll
 0000:fffdb000       .debug$S                   0000000180000000     ucrt:api-ms-win-crt-runtime-l1-1-0.dll
 0000:fffdb000       .debug$S                   0000000180000000     ucrt:api-ms-win-crt-runtime-l1-1-0.dll
 0000:fffdb000       .debug$S                   0000000180000000     ucrt:api-ms-win-crt-runtime-l1-1-0.dll
 0000:fffdb000       .debug$S                   0000000180000000     ucrt:api-ms-win-crt-runtime-l1-1-0.dll
 0000:fffdb000       .debug$S                   0000000180000000     ucrt:api-ms-win-crt-runtime-l1-1-0.dll
 0000:fffdb000       .debug$S                   0000000180000000     ucrt:api-ms-win-crt-runtime-l1-1-0.dll
 0000:fffdb000       .debug$S                   0000000180000000     ucrt:api-ms-win-crt-runtime-l1-1-0.dll
 0000:fffdb000       .debug$S                   0000000180000000     ucrt:api-ms-win-crt-runtime-l1-1-0.dll
 0000:fffdb000       .debug$S                   0000000180000000     ucrt:api-ms-win-crt-runtime-l1-1-0.dll
 0000:fffdb000       .debug$S                   0000000180000000     ucrt:api-ms-win-crt-runtime-l1-1-0.dll
 0000:fffdb000       .debug$S                   0000000180000000     ucrt:api-ms-win-crt-runtime-l1-1-0.dll
 0000:fffdb000       .debug$S                   0000000180000000     ucrt:api-ms-win-crt-runtime-l1-1-0.dll
 0000:fffdb000       .debug$S                   0000000180000000     ucrt:api-ms-win-crt-runtime-l1-1-0.dll
 0000:fffdb000       .debug$S                   0000000180000000     ucrt:api-ms-win-crt-runtime-l1-1-0.dll
 0000:fffdb000       .debug$S                   0000000180000000     ucrt:api-ms-win-crt-runtime-l1-1-0.dll
 0000:fffdb000       .debug$S                   0000000180000000     ucrt:api-ms-win-crt-runtime-l1-1-0.dll
 0000:fffdb000       .debug$S                   0000000180000000     ucrt:api-ms-win-crt-stdio-l1-1-0.dll
 0000:fffdb000       .debug$S                   0000000180000000     ucrt:api-ms-win-crt-stdio-l1-1-0.dll
 0000:fffdb000       .debug$S                   0000000180000000     ucrt:api-ms-win-crt-stdio-l1-1-0.dll
 0000:fffdb000       .debug$S                   0000000180000000     ucrt:api-ms-win-crt-stdio-l1-1-0.dll
 0000:fffdb000       .debug$S                   0000000180000000     ucrt:api-ms-win-crt-stdio-l1-1-0.dll
 0000:fffdb000       .debug$S                   0000000180000000     ucrt:api-ms-win-crt-stdio-l1-1-0.dll
 0000:fffdb000       .debug$S                   0000000180000000     ucrt:api-ms-win-crt-stdio-l1-1-0.dll
 0000:fffdb000       .debug$S                   0000000180000000     ucrt:api-ms-win-crt-stdio-l1-1-0.dll
 0000:fffdb000       .debug$S                   0000000180000000     ucrt:api-ms-win-crt-stdio-l1-1-0.dll
 0000:fffdb000       .debug$S                   0000000180000000     ucrt:api-ms-win-crt-stdio-l1-1-0.dll
 0000:fffdb000       .debug$S                   0000000180000000     ucrt:api-ms-win-crt-string-l1-1-0.dll
 0000:fffdb000       .debug$S                   0000000180000000     ucrt:api-ms-win-crt-string-l1-1-0.dll
 0000:fffdb000       .debug$S                   0000000180000000     ucrt:api-ms-win-crt-string-l1-1-0.dll
 0000:fffdb000       .debug$S                   0000000180000000     ucrt:api-ms-win-crt-string-l1-1-0.dll
 0000:fffdb000       .debug$S                   0000000180000000     ucrt:api-ms-win-crt-string-l1-1-0.dll
 0000:fffdb000       .debug$S                   0000000180000000     ucrt:api-ms-win-crt-string-l1-1-0.dll
 0000:fffdb000       .debug$S                   0000000180000000     ucrt:api-ms-win-crt-string-l1-1-0.dll
 0000:fffdb000       .debug$S                   0000000180000000     ucrt:api-ms-win-crt-string-l1-1-0.dll
 0000:fffdb000       .debug$S                   0000000180000000     kernel32:KERNEL32.dll
 0000:fffdb000       .debug$S                   0000000180000000     kernel32:KERNEL32.dll
 0000:fffdb000       .debug$S                   0000000180000000     kernel32:KERNEL32.dll
 0000:fffdb000       .debug$S                   0000000180000000     kernel32:KERNEL32.dll
 0000:fffdb000       .debug$S                   0000000180000000     kernel32:KERNEL32.dll
 0000:fffdb000       .debug$S                   0000000180000000     kernel32:KERNEL32.dll
 0000:fffdb000       .debug$S                   0000000180000000     kernel32:KERNEL32.dll
 0000:fffdb000       .debug$S                   0000000180000000     kernel32:KERNEL32.dll
 0000:fffdb000       .debug$S                   0000000180000000     kernel32:KERNEL32.dll
 0000:fffdb000       .debug$S                   0000000180000000     kernel32:KERNEL32.dll
 0000:fffdb000       .debug$S                   0000000180000000     kernel32:KERNEL32.dll
 0000:fffdb000       .debug$S                   0000000180000000     kernel32:KERNEL32.dll
 0000:fffdb000       .debug$S                   0000000180000000     kernel32:KERNEL32.dll
 0000:fffdb000       .debug$S                   0000000180000000     kernel32:KERNEL32.dll
 0000:fffdb000       .debug$S                   0000000180000000     kernel32:KERNEL32.dll
 0000:fffdb000       .debug$S                   0000000180000000     kernel32:KERNEL32.dll
 0000:fffdb000       .debug$S                   0000000180000000     kernel32:KERNEL32.dll
 0000:fffdb000       .debug$S                   0000000180000000     kernel32:KERNEL32.dll
 0000:fffdb000       .debug$S                   0000000180000000     kernel32:KERNEL32.dll
 0000:fffdb000       .debug$S                   0000000180000000     kernel32:KERNEL32.dll
 0000:fffdb000       .debug$S                   0000000180000000     kernel32:KERNEL32.dll
 0000:fffdb000       .debug$S                   0000000180000000     kernel32:KERNEL32.dll
 0000:fffdb000       .debug$S                   0000000180000000     kernel32:KERNEL32.dll
 0000:fffdb000       .debug$S                   0000000180000000     kernel32:KERNEL32.dll
 0000:fffdb000       .debug$S                   0000000180000000     kernel32:KERNEL32.dll
 0000:fffdb000       .debug$S                   0000000180000000     kernel32:KERNEL32.dll
 0000:fffdb000       .debug$S                   0000000180000000     kernel32:KERNEL32.dll
 0000:fffdb000       .debug$S                   0000000180000000     kernel32:KERNEL32.dll
 0001:00000e74       addRefToVerify             0000000180001e74 f   libgetfldecl004.obj
 0001:00000ee0       agentThreadWrapper         0000000180001ee0 f   libgetfldecl004.obj
 0001:000010d0       file_basename              00000001800020d0 f   libgetfldecl004.obj
 0001:0000173c       startAgentThreadWrapper    000000018000273c f   libgetfldecl004.obj
 0001:00001a7c       syncDebuggeeStatus         0000000180002a7c f   libgetfldecl004.obj
 0001:00001d1c       capture_previous_context   0000000180002d1c f   MSVCRT:gs_report.obj
 0001:00001d90       ?__scrt_initialize_thread_safe_statics@@YAHXZ 0000000180002d90 f   MSVCRT:thread_safe_statics.obj
 0001:00001e60       ?__scrt_uninitialize_thread_safe_statics@@YAXXZ 0000000180002e60 f   MSVCRT:thread_safe_statics.obj
 0001:00001f10       $$000000                   0000000180002f10     MSVCRT:amdsecgs.obj
 0001:00001f40       ?dllmain_crt_dispatch@@YAHQEAUHINSTANCE__@@KQEAX@Z 0000000180002f40 f   MSVCRT:dll_dllmain.obj
 0001:00001f90       ?dllmain_crt_process_attach@@YAHQEAUHINSTANCE__@@QEAX@Z 0000000180002f90 f   MSVCRT:dll_dllmain.obj
 0001:000020a8       ?dllmain_crt_process_detach@@YAH_N@Z 00000001800030a8 f   MSVCRT:dll_dllmain.obj
 0001:0000212c       ?dllmain_dispatch@@YAHQEAUHINSTANCE__@@KQEAX@Z 000000018000312c f   MSVCRT:dll_dllmain.obj
 0001:00002b40       $$000000                   0000000180003b40     MSVCRT:guard_dispatch.obj
 0001:00002b60       $$000000                   0000000180003b60     MSVCRT:guard_xfg_dispatch.obj
 0001:00002b76       ?fin$0@?0??dllmain_crt_process_attach@@YAHQEAUHINSTANCE__@@QEAX@Z@4HA 0000000180003b76 f   MSVCRT:dll_dllmain.obj
 0001:00002b8d       ?fin$0@?0??dllmain_crt_process_detach@@YAH_N@Z@4HA 0000000180003b8d f   MSVCRT:dll_dllmain.obj
 0001:00002ba6       ?fin$1@?0??dllmain_crt_process_detach@@YAH_N@Z@4HA 0000000180003ba6 f   MSVCRT:dll_dllmain.obj
 0001:00002bba       ?filt$0@?0??dllmain_dispatch@@YAHQEAUHINSTANCE__@@KQEAX@Z@4HA 0000000180003bba f   MSVCRT:dll_dllmain.obj
 0001:00002bf0       __scrt_is_nonwritable_in_current_image$filt$0 0000000180003bf0 f   MSVCRT:utility.obj
 0002:000001e8       ?__scrt_initialize_tss_var@@3P6AHXZEA 00000001800041e8     MSVCRT:thread_safe_statics.obj
 0002:00000310       ?opcLengths@@3QBEB         0000000180004310     libgetfldecl004.obj
 0002:00001b18       GS_ExceptionPointers       0000000180005b18     MSVCRT:gs_report.obj
 0002:00002218       $unwind$fprintf            0000000180006218     libgetfldecl004.obj
 0002:00002224       $unwind$printf             0000000180006224     libgetfldecl004.obj
 0002:00002230       $unwind$?NewObject@JNIEnv_@@QEAAPEAV_jobject@@PEAV_jclass@@PEAU_jmethodID@@ZZ 0000000180006230     libgetfldecl004.obj
 0002:00002230       $unwind$nsk_lcomplain      0000000180006230     libgetfldecl004.obj
 0002:00002230       $unwind$nsk_ldisplay       0000000180006230     libgetfldecl004.obj
 0002:00002238       $unwind$nsk_lvdisplay      0000000180006238     libgetfldecl004.obj
 0002:00002238       $unwind$_RTC_Initialize    0000000180006238     MSVCRT:initsect.obj
 0002:00002238       $unwind$_RTC_Terminate     0000000180006238     MSVCRT:initsect.obj
 0002:00002238       $unwind$?__scrt_initialize_thread_safe_statics@@YAHXZ 0000000180006238     MSVCRT:thread_safe_statics.obj
 0002:00002244       $unwind$nsk_lvcomplain     0000000180006244     libgetfldecl004.obj
 0002:0000225c       $unwind$nsk_ltrace         000000018000625c     libgetfldecl004.obj
 0002:0000225c       $unwind$__report_gsfailure 000000018000625c     MSVCRT:gs_report.obj
 0002:00002264       $unwind$Agent_Initialize   0000000180006264     libgetfldecl004.obj
 0002:00002264       $unwind$nsk_lvtrace        0000000180006264     libgetfldecl004.obj
 0002:00002264       $unwind$__raise_securityfailure 0000000180006264     MSVCRT:gs_report.obj
 0002:00002264       $unwind$__scrt_initialize_crt 0000000180006264     MSVCRT:utility.obj
 0002:00002264       $unwind$__scrt_initialize_onexit_tables 0000000180006264     MSVCRT:utility.obj
 0002:00002264       $unwind$__scrt_release_startup_lock 0000000180006264     MSVCRT:utility.obj
 0002:00002264       $unwind$__scrt_uninitialize_crt 0000000180006264     MSVCRT:utility.obj
 0002:00002264       $unwind$_onexit            0000000180006264     MSVCRT:utility.obj
 0002:0000226c       $unwind$nsk_lverify        000000018000626c     libgetfldecl004.obj
 0002:0000227c       $unwind$nsk_vprintf        000000018000627c     libgetfldecl004.obj
 0002:0000228c       $unwind$nsk_printf         000000018000628c     libgetfldecl004.obj
 0002:00002294       $unwind$?nsk_jni_lverify@@YAHHPEAUJNIEnv_@@HQEBDH1ZZ 0000000180006294     libgetfldecl004.obj
 0002:000022a8       $unwind$?nsk_jni_check_exception@@YAHPEAUJNIEnv_@@QEBDH@Z 00000001800062a8     libgetfldecl004.obj
 0002:000022c4       $unwind$Java_nsk_jvmti_unit_FollowReferences_FollowRefObjects_resetTags 00000001800062c4     libgetfldecl004.obj
 0002:000022c4       $unwind$addRefToVerify     00000001800062c4     libgetfldecl004.obj
 0002:000022c4       $unwind$nsk_jvmti_resetAgentData 00000001800062c4     libgetfldecl004.obj
 0002:000022c4       $unwind$nsk_jvmti_setFailStatus 00000001800062c4     libgetfldecl004.obj
 0002:000022c4       $unwind$__scrt_initialize_default_local_stdio_options 00000001800062c4     MSVCRT:default_local_stdio_options.obj
 0002:000022c4       $unwind$?dllmain_crt_dispatch@@YAHQEAUHINSTANCE__@@KQEAX@Z 00000001800062c4     MSVCRT:dll_dllmain.obj
 0002:000022c4       $unwind$DllMain            00000001800062c4     MSVCRT:dll_dllmain_stub.obj
 0002:000022c4       $unwind$__GSHandlerCheck   00000001800062c4     MSVCRT:gshandler.obj
 0002:000022c4       $unwind$?__scrt_uninitialize_thread_safe_statics@@YAXXZ 00000001800062c4     MSVCRT:thread_safe_statics.obj
 0002:000022c4       $unwind$__scrt_acquire_startup_lock 00000001800062c4     MSVCRT:utility.obj
 0002:000022c4       $unwind$__scrt_dllmain_after_initialize_c 00000001800062c4     MSVCRT:utility.obj
 0002:000022c4       $unwind$__scrt_dllmain_before_initialize_c 00000001800062c4     MSVCRT:utility.obj
 0002:000022c4       $unwind$__scrt_dllmain_crt_thread_attach 00000001800062c4     MSVCRT:utility.obj
 0002:000022c4       $unwind$__scrt_dllmain_crt_thread_detach 00000001800062c4     MSVCRT:utility.obj
 0002:000022c4       $unwind$__scrt_dllmain_uninitialize_c 00000001800062c4     MSVCRT:utility.obj
 0002:000022c4       $unwind$__scrt_dllmain_uninitialize_critical 00000001800062c4     MSVCRT:utility.obj
 0002:000022c4       $unwind$atexit             00000001800062c4     MSVCRT:utility.obj
 0002:000022cc       $unwind$nsk_jvmti_lverify  00000001800062cc     libgetfldecl004.obj
 0002:000022e0       $unwind$exitOnError        00000001800062e0     libgetfldecl004.obj
 0002:000022f0       $unwind$Java_nsk_share_jvmti_ArgumentHandler_getAgentOptionsString 00000001800062f0     libgetfldecl004.obj
 0002:00002304       $unwind$Java_nsk_jvmti_unit_FollowReferences_FollowRefObjects_getTag 0000000180006304     libgetfldecl004.obj
 0002:00002304       $unwind$Java_nsk_share_jvmti_DebugeeClass_checkStatus 0000000180006304     libgetfldecl004.obj
 0002:00002304       $unwind$agentThreadWrapper 0000000180006304     libgetfldecl004.obj
 0002:00002314       $unwind$startAgentThreadWrapper 0000000180006314     libgetfldecl004.obj
 0002:00002330       $unwind$syncDebuggeeStatus 0000000180006330     libgetfldecl004.obj
 0002:00002330       $unwind$__scrt_dllmain_exception_filter 0000000180006330     MSVCRT:utility.obj
 0002:00002344       $unwind$Java_nsk_share_jvmti_DebugeeClass_resetAgentData 0000000180006344     libgetfldecl004.obj
 0002:0000234c       $unwind$MA_checkStatus     000000018000634c     libgetfldecl004.obj
 0002:00002360       $unwind$Java_nsk_jvmti_unit_FollowReferences_FollowRefObjects_setTag 0000000180006360     libgetfldecl004.obj
 0002:00002378       $unwind$Java_nsk_jvmti_unit_FollowReferences_FollowRefObjects_addRefToVerify 0000000180006378     libgetfldecl004.obj
 0002:00002394       $unwind$Java_nsk_jvmti_GetFieldDeclaringClass_getfldecl004_check 0000000180006394     libgetfldecl004.obj
 0002:000023ac       $unwind$capture_previous_context 00000001800063ac     MSVCRT:gs_report.obj
 0002:000023b8       $unwind$__GSHandlerCheckCommon 00000001800063b8     MSVCRT:gshandler.obj
 0002:000023c0       $xdatasym                  00000001800063c0     MSVCRT:amdsecgs.obj
 0002:000023c4       $unwind$?dllmain_crt_process_attach@@YAHQEAUHINSTANCE__@@QEAX@Z 00000001800063c4     MSVCRT:dll_dllmain.obj
 0002:00002400       $unwind$?fin$0@?0??dllmain_crt_process_attach@@YAHQEAUHINSTANCE__@@QEAX@Z@4HA 0000000180006400     MSVCRT:dll_dllmain.obj
 0002:00002400       $unwind$?fin$0@?0??dllmain_crt_process_detach@@YAH_N@Z@4HA 0000000180006400     MSVCRT:dll_dllmain.obj
 0002:00002400       $unwind$?fin$1@?0??dllmain_crt_process_detach@@YAH_N@Z@4HA 0000000180006400     MSVCRT:dll_dllmain.obj
 0002:00002408       $unwind$?dllmain_crt_process_detach@@YAH_N@Z 0000000180006408     MSVCRT:dll_dllmain.obj
 0002:0000245c       $unwind$?dllmain_dispatch@@YAHQEAUHINSTANCE__@@KQEAX@Z 000000018000645c     MSVCRT:dll_dllmain.obj
 0002:00002484       $unwind$?filt$0@?0??dllmain_dispatch@@YAHQEAUHINSTANCE__@@KQEAX@Z@4HA 0000000180006484     MSVCRT:dll_dllmain.obj
 0002:0000248c       $unwind$_DllMainCRTStartup 000000018000648c     MSVCRT:dll_dllmain.obj
 0002:0000249c       $unwind$__scrt_is_nonwritable_in_current_image 000000018000649c     MSVCRT:utility.obj
 0002:000024bc       $unwind$__scrt_is_nonwritable_in_current_image$filt$0 00000001800064bc     MSVCRT:utility.obj
 0002:000024c4       $unwind$__scrt_fastfail    00000001800064c4     MSVCRT:utility_desktop.obj
 0002:000024d4       $unwind$__security_init_cookie 00000001800064d4     MSVCRT:gs_support.obj
 0002:000024e0       $unwind$__isa_available_init 00000001800064e0     MSVCRT:cpu_disp.obj
 0002:000024f0       $xdatasym                  00000001800064f0     MSVCRT:guard_dispatch.obj
 0002:000024f8       $xdatasym                  00000001800064f8     MSVCRT:guard_xfg_dispatch.obj
 0002:00002500       .edata                     0000000180006500     getfldecl004.exp
 0002:00002528       rgpv                       0000000180006528     getfldecl004.exp
 0002:00002568       rgszName                   0000000180006568     getfldecl004.exp
 0002:000025a8       rgwOrd                     00000001800065a8     getfldecl004.exp
 0002:000025c8       szName                     00000001800065c8     getfldecl004.exp
 0002:000025d9       $N00001                    00000001800065d9     getfldecl004.exp
 0002:000025e8       $N00002                    00000001800065e8     getfldecl004.exp
 0002:000025f5       $N00003                    00000001800065f5     getfldecl004.exp
 0002:0000262e       $N00004                    000000018000662e     getfldecl004.exp
 0002:00002668       $N00005                    0000000180006668     getfldecl004.exp
 0002:000026ad       $N00006                    00000001800066ad     getfldecl004.exp
 0002:000026ea       $N00007                    00000001800066ea     getfldecl004.exp
 0002:00002732       $N00008                    0000000180006732     getfldecl004.exp
 0002:00002772       $N00009                    0000000180006772     getfldecl004.exp
 0002:000027af       $N00010                    00000001800067af     getfldecl004.exp
 0002:000027ea       $N00011                    00000001800067ea     getfldecl004.exp
 0002:00002818       $N00012                    0000000180006818     getfldecl004.exp
 0002:00002849       $N00013                    0000000180006849     getfldecl004.exp
 0002:00002878       $N00014                    0000000180006878     getfldecl004.exp
 0002:000028a7       $N00015                    00000001800068a7     getfldecl004.exp
 0002:000028dc       $N00016                    00000001800068dc     getfldecl004.exp
 0002:00002cea       .idata$6                   0000000180006cea     kernel32:KERNEL32.dll
 0002:00002d4e       .idata$6                   0000000180006d4e     vcruntime:VCRUNTIME140.dll
 0002:00002eba       .idata$6                   0000000180006eba     ucrt:api-ms-win-crt-runtime-l1-1-0.dll
 0002:00002edc       .idata$6                   0000000180006edc     ucrt:api-ms-win-crt-stdio-l1-1-0.dll
 0002:00002efc       .idata$6                   0000000180006efc     ucrt:api-ms-win-crt-string-l1-1-0.dll
 0003:00000000       ?codeAttributeName@@3PEBDEB 0000000180007000     libgetfldecl004.obj
 0003:00000008       ?lineNumberAttributeName@@3PEBDEB 0000000180007008     libgetfldecl004.obj
 0003:00000010       ?localVarAttributeName@@3PEBDEB 0000000180007010     libgetfldecl004.obj
 0003:00000018       ?localVarTypeAttributeName@@3PEBDEB 0000000180007018     libgetfldecl004.obj
 0003:00000020       ?stackMapAttributeName@@3PEBDEB 0000000180007020     libgetfldecl004.obj
 0003:00000028       ?callBytes@@3PAEA          0000000180007028     libgetfldecl004.obj
 0003:0000002c       ?allocBytes@@3PAEA         000000018000702c     libgetfldecl004.obj
 0003:00000030       fields                     0000000180007030     libgetfldecl004.obj
 0003:0001abf4       redefineAttempted          0000000180021bf4     libgetfldecl004.obj
 0003:0001abf8       nsk_context                0000000180021bf8     libgetfldecl004.obj
 0003:0001ac04       redefineSucceed            0000000180021c04     libgetfldecl004.obj
 0003:0001ac08       agentFailed                0000000180021c08     libgetfldecl004.obj
 0003:0001ac0c       currentAgentStatus         0000000180021c0c     libgetfldecl004.obj
 0003:0001ac10       context                    0000000180021c10     libgetfldecl004.obj
 0003:0001acc8       agentThread                0000000180021cc8     libgetfldecl004.obj
 0003:0001acd0       agentThreadProc            0000000180021cd0     libgetfldecl004.obj
 0003:0001acd8       agentThreadArg             0000000180021cd8     libgetfldecl004.obj
 0003:0001ace0       agent_data                 0000000180021ce0     libgetfldecl004.obj
 0003:0001acf0       jvmti_env                  0000000180021cf0     libgetfldecl004.obj
 0003:0001acf8       jvm                        0000000180021cf8     libgetfldecl004.obj
 0003:0001ad00       jni_env                    0000000180021d00     libgetfldecl004.obj
 0003:0001ad08       checkStatus_func           0000000180021d08     libgetfldecl004.obj
 0003:0001ad10       ?codeAttributeIndex@@3GA   0000000180021d10     libgetfldecl004.obj
 0003:0001ad12       printdump                  0000000180021d12     libgetfldecl004.obj
 0003:0001ad14       ?lineNumberAttributeIndex@@3GA 0000000180021d14     libgetfldecl004.obj
 0003:0001ad18       ?localVarAttributeIndex@@3GA 0000000180021d18     libgetfldecl004.obj
 0003:0001ad1c       ?localVarTypeAttributeIndex@@3GA 0000000180021d1c     libgetfldecl004.obj
 0003:0001ad20       ?stackMapAttributeIndex@@3GA 0000000180021d20     libgetfldecl004.obj
 0003:0001ad24       ?stackFrameOffset@@3GA     0000000180021d24     libgetfldecl004.obj
 0003:0001ad28       ?mode@@3HA                 0000000180021d28     libgetfldecl004.obj
 0003:0001ad2c       ?constantPoolSize@@3GA     0000000180021d2c     libgetfldecl004.obj
 0003:0001ad30       ?orig@@3PEBEEB             0000000180021d30     libgetfldecl004.obj
 0003:0001ad38       ?gen@@3PEAEEA              0000000180021d38     libgetfldecl004.obj
 0003:0001ad40       ?inputPos@@3PEAEEA         0000000180021d40     libgetfldecl004.obj
 0003:0001ad48       ?endPos@@3PEBEEB           0000000180021d48     libgetfldecl004.obj
 0003:0001ad50       ?genPos@@3PEAEEA           0000000180021d50     libgetfldecl004.obj
 0003:0001ad58       ?markPos@@3PEAEEA          0000000180021d58     libgetfldecl004.obj
 0003:0001ad60       ?constantPool@@3PEAPEADEA  0000000180021d60     libgetfldecl004.obj
 0003:0001ad68       ?constantPoolCount@@3GA    0000000180021d68     libgetfldecl004.obj
 0003:0001ad6c       ?zeroBytes@@3PAEA          0000000180021d6c     libgetfldecl004.obj
 0003:0001ad70       ?codeLength@@3IA           0000000180021d70     libgetfldecl004.obj
 0003:0001ad74       result                     0000000180021d74     libgetfldecl004.obj
 0003:0001ad78       ?map@@3PEAIEA              0000000180021d78     libgetfldecl004.obj
 0003:0001ad80       ?widening@@3PEACEA         0000000180021d80     libgetfldecl004.obj
 0003:0001ad88       jvmti                      0000000180021d88     libgetfldecl004.obj
 0003:0001ada0       GS_ExceptionRecord         0000000180021da0     MSVCRT:gs_report.obj
 0003:0001ae40       GS_ContextRecord           0000000180021e40     MSVCRT:gs_report.obj
 0003:0001b310       ?g_tss_cv@@3U_RTL_CONDITION_VARIABLE@@A 0000000180022310     MSVCRT:thread_safe_statics.obj
 0003:0001b318       ?g_tss_event@@3PEAXEA      0000000180022318     MSVCRT:thread_safe_statics.obj
 0003:0001b320       ?g_tss_mutex@@3U_RTL_CRITICAL_SECTION@@A 0000000180022320     MSVCRT:thread_safe_statics.obj
 0003:0001b348       ?g_sleep_condition_variable_cs@@3P6AHPEAU_RTL_CONDITION_VARIABLE@@PEAU_RTL_CRITICAL_SECTION@@K@ZEA 0000000180022348     MSVCRT:thread_safe_statics.obj
 0003:0001b350       ?g_wake_all_condition_variable@@3P6AXPEAU_RTL_CONDITION_VARIABLE@@@ZEA 0000000180022350     MSVCRT:thread_safe_statics.obj
 0003:0001b35c       ?__proc_attached@@3HA      000000018002235c     MSVCRT:dll_dllmain.obj
 0003:0001b370       ?is_initialized_as_dll@@3_NA 0000000180022370     MSVCRT:utility.obj
 0003:0001b371       ?module_local_atexit_table_initialized@@3_NA 0000000180022371     MSVCRT:utility.obj
 0003:0001b378       ?module_local_atexit_table@@3U_onexit_table_t@@A 0000000180022378     MSVCRT:utility.obj
 0003:0001b390       ?module_local_at_quick_exit_table@@3U_onexit_table_t@@A 0000000180022390     MSVCRT:utility.obj
